
04_gpio_input.elf:     file format elf32-littlearm

Sections:
Idx Name          Size      VMA       LMA       File off  Algn
  0 .isr_vector   00000198  08000000  08000000  00010000  2**0
                  CONTENTS, ALLOC, LOAD, READONLY, DATA
  1 .text         00000174  08000198  08000198  00010198  2**2
                  CONTENTS, ALLOC, LOAD, READONLY, CODE
  2 .rodata       00000000  0800030c  08000314  00010314  2**0
                  CONTENTS, ALLOC, LOAD, DATA
  3 .ARM.extab    00000000  0800030c  0800030c  00010314  2**0
                  CONTENTS
  4 .ARM          00000000  0800030c  0800030c  00010314  2**0
                  CONTENTS
  5 .preinit_array 00000000  0800030c  08000314  00010314  2**0
                  CONTENTS, ALLOC, LOAD, DATA
  6 .init_array   00000004  0800030c  0800030c  0001030c  2**2
                  CONTENTS, ALLOC, LOAD, DATA
  7 .fini_array   00000004  08000310  08000310  00010310  2**2
                  CONTENTS, ALLOC, LOAD, DATA
  8 .data         00000000  20000000  20000000  00010314  2**0
                  CONTENTS, ALLOC, LOAD, DATA
  9 .bss          0000001c  20000000  08000314  00020000  2**2
                  ALLOC
 10 ._user_heap_stack 00000604  2000001c  08000314  0002001c  2**0
                  ALLOC
 11 .ARM.attributes 00000030  00000000  00000000  00010314  2**0
                  CONTENTS, READONLY
 12 .debug_info   000003fc  00000000  00000000  00010344  2**0
                  CONTENTS, READONLY, DEBUGGING, OCTETS
 13 .debug_abbrev 000000f0  00000000  00000000  00010740  2**0
                  CONTENTS, READONLY, DEBUGGING, OCTETS
 14 .debug_aranges 00000048  00000000  00000000  00010830  2**3
                  CONTENTS, READONLY, DEBUGGING, OCTETS
 15 .debug_ranges 00000030  00000000  00000000  00010878  2**3
                  CONTENTS, READONLY, DEBUGGING, OCTETS
 16 .debug_macro  0000dc2c  00000000  00000000  000108a8  2**0
                  CONTENTS, READONLY, DEBUGGING, OCTETS
 17 .debug_line   00000545  00000000  00000000  0001e4d4  2**0
                  CONTENTS, READONLY, DEBUGGING, OCTETS
 18 .debug_str    0004f6c9  00000000  00000000  0001ea19  2**0
                  CONTENTS, READONLY, DEBUGGING, OCTETS
 19 .comment      00000053  00000000  00000000  0006e0e2  2**0
                  CONTENTS, READONLY
 20 .debug_frame  00000054  00000000  00000000  0006e138  2**2
                  CONTENTS, READONLY, DEBUGGING, OCTETS

Disassembly of section .text:

08000198 <__do_global_dtors_aux>:
 8000198:	b510      	push	{r4, lr}
 800019a:	4c05      	ldr	r4, [pc, #20]	; (80001b0 <__do_global_dtors_aux+0x18>)
 800019c:	7823      	ldrb	r3, [r4, #0]
 800019e:	b933      	cbnz	r3, 80001ae <__do_global_dtors_aux+0x16>
 80001a0:	4b04      	ldr	r3, [pc, #16]	; (80001b4 <__do_global_dtors_aux+0x1c>)
 80001a2:	b113      	cbz	r3, 80001aa <__do_global_dtors_aux+0x12>
 80001a4:	4804      	ldr	r0, [pc, #16]	; (80001b8 <__do_global_dtors_aux+0x20>)
 80001a6:	f3af 8000 	nop.w
 80001aa:	2301      	movs	r3, #1
 80001ac:	7023      	strb	r3, [r4, #0]
 80001ae:	bd10      	pop	{r4, pc}
 80001b0:	20000000 	.word	0x20000000
 80001b4:	00000000 	.word	0x00000000
 80001b8:	080002f4 	.word	0x080002f4

080001bc <frame_dummy>:
 80001bc:	b508      	push	{r3, lr}
 80001be:	4b03      	ldr	r3, [pc, #12]	; (80001cc <frame_dummy+0x10>)
 80001c0:	b11b      	cbz	r3, 80001ca <frame_dummy+0xe>
 80001c2:	4903      	ldr	r1, [pc, #12]	; (80001d0 <frame_dummy+0x14>)
 80001c4:	4803      	ldr	r0, [pc, #12]	; (80001d4 <frame_dummy+0x18>)
 80001c6:	f3af 8000 	nop.w
 80001ca:	bd08      	pop	{r3, pc}
 80001cc:	00000000 	.word	0x00000000
 80001d0:	20000004 	.word	0x20000004
 80001d4:	080002f4 	.word	0x080002f4

080001d8 <main>:
#define PIN13 (1U<<13)

#define LED_PIN PIN5
#define BTN_PIN PIN13

int main(void){
 80001d8:	b480      	push	{r7}
 80001da:	af00      	add	r7, sp, #0
	/* Enable clock access to GPIOA and GPIOC */
	RCC->AHB1ENR |= GPIOAEN;
 80001dc:	4b1b      	ldr	r3, [pc, #108]	; (800024c <main+0x74>)
 80001de:	6b1b      	ldr	r3, [r3, #48]	; 0x30
 80001e0:	4a1a      	ldr	r2, [pc, #104]	; (800024c <main+0x74>)
 80001e2:	f043 0301 	orr.w	r3, r3, #1
 80001e6:	6313      	str	r3, [r2, #48]	; 0x30
	RCC->AHB1ENR |= GPIOCEN;
 80001e8:	4b18      	ldr	r3, [pc, #96]	; (800024c <main+0x74>)
 80001ea:	6b1b      	ldr	r3, [r3, #48]	; 0x30
 80001ec:	4a17      	ldr	r2, [pc, #92]	; (800024c <main+0x74>)
 80001ee:	f043 0304 	orr.w	r3, r3, #4
 80001f2:	6313      	str	r3, [r2, #48]	; 0x30

	/*Set PA5 as output pin*/
	GPIOA->MODER |= (1U<<10);
 80001f4:	4b16      	ldr	r3, [pc, #88]	; (8000250 <main+0x78>)
 80001f6:	681b      	ldr	r3, [r3, #0]
 80001f8:	4a15      	ldr	r2, [pc, #84]	; (8000250 <main+0x78>)
 80001fa:	f443 6380 	orr.w	r3, r3, #1024	; 0x400
 80001fe:	6013      	str	r3, [r2, #0]
	GPIOA->MODER &=~ (1U<<11);
 8000200:	4b13      	ldr	r3, [pc, #76]	; (8000250 <main+0x78>)
 8000202:	681b      	ldr	r3, [r3, #0]
 8000204:	4a12      	ldr	r2, [pc, #72]	; (8000250 <main+0x78>)
 8000206:	f423 6300 	bic.w	r3, r3, #2048	; 0x800
 800020a:	6013      	str	r3, [r2, #0]

	/*Set PC13 as input pin*/
	GPIOC->MODER &=~ (1U<<26);
 800020c:	4b11      	ldr	r3, [pc, #68]	; (8000254 <main+0x7c>)
 800020e:	681b      	ldr	r3, [r3, #0]
 8000210:	4a10      	ldr	r2, [pc, #64]	; (8000254 <main+0x7c>)
 8000212:	f023 6380 	bic.w	r3, r3, #67108864	; 0x4000000
 8000216:	6013      	str	r3, [r2, #0]
	GPIOC->MODER &=~ (1U<<27);
 8000218:	4b0e      	ldr	r3, [pc, #56]	; (8000254 <main+0x7c>)
 800021a:	681b      	ldr	r3, [r3, #0]
 800021c:	4a0d      	ldr	r2, [pc, #52]	; (8000254 <main+0x7c>)
 800021e:	f023 6300 	bic.w	r3, r3, #134217728	; 0x8000000
 8000222:	6013      	str	r3, [r2, #0]


	while (1){

		if(GPIOC->IDR & BTN_PIN){
 8000224:	4b0b      	ldr	r3, [pc, #44]	; (8000254 <main+0x7c>)
 8000226:	691b      	ldr	r3, [r3, #16]
 8000228:	f403 5300 	and.w	r3, r3, #8192	; 0x2000
 800022c:	2b00      	cmp	r3, #0
 800022e:	d006      	beq.n	800023e <main+0x66>
		GPIOA->BSRR ^=LED_PIN;
 8000230:	4b07      	ldr	r3, [pc, #28]	; (8000250 <main+0x78>)
 8000232:	699b      	ldr	r3, [r3, #24]
 8000234:	4a06      	ldr	r2, [pc, #24]	; (8000250 <main+0x78>)
 8000236:	f083 0320 	eor.w	r3, r3, #32
 800023a:	6193      	str	r3, [r2, #24]
 800023c:	e7f2      	b.n	8000224 <main+0x4c>
		}
		else{
		GPIOA->BSRR ^=(1U<<21);
 800023e:	4b04      	ldr	r3, [pc, #16]	; (8000250 <main+0x78>)
 8000240:	699b      	ldr	r3, [r3, #24]
 8000242:	4a03      	ldr	r2, [pc, #12]	; (8000250 <main+0x78>)
 8000244:	f483 1300 	eor.w	r3, r3, #2097152	; 0x200000
 8000248:	6193      	str	r3, [r2, #24]
		if(GPIOC->IDR & BTN_PIN){
 800024a:	e7eb      	b.n	8000224 <main+0x4c>
 800024c:	40023800 	.word	0x40023800
 8000250:	40020000 	.word	0x40020000
 8000254:	40020800 	.word	0x40020800

08000258 <Reset_Handler>:

  .section .text.Reset_Handler
  .weak Reset_Handler
  .type Reset_Handler, %function
Reset_Handler:
  ldr   r0, =_estack
 8000258:	480d      	ldr	r0, [pc, #52]	; (8000290 <LoopForever+0x2>)
  mov   sp, r0          /* set stack pointer */
 800025a:	4685      	mov	sp, r0
/* Call the clock system intitialization function.*/
  bl  SystemInit
 800025c:	f3af 8000 	nop.w

/* Copy the data segment initializers from flash to SRAM */
  ldr r0, =_sdata
 8000260:	480c      	ldr	r0, [pc, #48]	; (8000294 <LoopForever+0x6>)
  ldr r1, =_edata
 8000262:	490d      	ldr	r1, [pc, #52]	; (8000298 <LoopForever+0xa>)
  ldr r2, =_sidata
 8000264:	4a0d      	ldr	r2, [pc, #52]	; (800029c <LoopForever+0xe>)
  movs r3, #0
 8000266:	2300      	movs	r3, #0
  b LoopCopyDataInit
 8000268:	e002      	b.n	8000270 <LoopCopyDataInit>

0800026a <CopyDataInit>:

CopyDataInit:
  ldr r4, [r2, r3]
 800026a:	58d4      	ldr	r4, [r2, r3]
  str r4, [r0, r3]
 800026c:	50c4      	str	r4, [r0, r3]
  adds r3, r3, #4
 800026e:	3304      	adds	r3, #4

08000270 <LoopCopyDataInit>:

LoopCopyDataInit:
  adds r4, r0, r3
 8000270:	18c4      	adds	r4, r0, r3
  cmp r4, r1
 8000272:	428c      	cmp	r4, r1
  bcc CopyDataInit
 8000274:	d3f9      	bcc.n	800026a <CopyDataInit>

/* Zero fill the bss segment. */
  ldr r2, =_sbss
 8000276:	4a0a      	ldr	r2, [pc, #40]	; (80002a0 <LoopForever+0x12>)
  ldr r4, =_ebss
 8000278:	4c0a      	ldr	r4, [pc, #40]	; (80002a4 <LoopForever+0x16>)
  movs r3, #0
 800027a:	2300      	movs	r3, #0
  b LoopFillZerobss
 800027c:	e001      	b.n	8000282 <LoopFillZerobss>

0800027e <FillZerobss>:

FillZerobss:
  str  r3, [r2]
 800027e:	6013      	str	r3, [r2, #0]
  adds r2, r2, #4
 8000280:	3204      	adds	r2, #4

08000282 <LoopFillZerobss>:

LoopFillZerobss:
  cmp r2, r4
 8000282:	42a2      	cmp	r2, r4
  bcc FillZerobss
 8000284:	d3fb      	bcc.n	800027e <FillZerobss>

/* Call static constructors */
  bl __libc_init_array
 8000286:	f000 f811 	bl	80002ac <__libc_init_array>
/* Call the application's entry point.*/
  bl main
 800028a:	f7ff ffa5 	bl	80001d8 <main>

0800028e <LoopForever>:

LoopForever:
    b LoopForever
 800028e:	e7fe      	b.n	800028e <LoopForever>
  ldr   r0, =_estack
 8000290:	20020000 	.word	0x20020000
  ldr r0, =_sdata
 8000294:	20000000 	.word	0x20000000
  ldr r1, =_edata
 8000298:	20000000 	.word	0x20000000
  ldr r2, =_sidata
 800029c:	08000314 	.word	0x08000314
  ldr r2, =_sbss
 80002a0:	20000000 	.word	0x20000000
  ldr r4, =_ebss
 80002a4:	2000001c 	.word	0x2000001c

080002a8 <ADC_IRQHandler>:
 * @retval : None
*/
  .section .text.Default_Handler,"ax",%progbits
Default_Handler:
Infinite_Loop:
  b Infinite_Loop
 80002a8:	e7fe      	b.n	80002a8 <ADC_IRQHandler>
	...

080002ac <__libc_init_array>:
 80002ac:	b570      	push	{r4, r5, r6, lr}
 80002ae:	4d0d      	ldr	r5, [pc, #52]	; (80002e4 <__libc_init_array+0x38>)
 80002b0:	4c0d      	ldr	r4, [pc, #52]	; (80002e8 <__libc_init_array+0x3c>)
 80002b2:	1b64      	subs	r4, r4, r5
 80002b4:	10a4      	asrs	r4, r4, #2
 80002b6:	2600      	movs	r6, #0
 80002b8:	42a6      	cmp	r6, r4
 80002ba:	d109      	bne.n	80002d0 <__libc_init_array+0x24>
 80002bc:	4d0b      	ldr	r5, [pc, #44]	; (80002ec <__libc_init_array+0x40>)
 80002be:	4c0c      	ldr	r4, [pc, #48]	; (80002f0 <__libc_init_array+0x44>)
 80002c0:	f000 f818 	bl	80002f4 <_init>
 80002c4:	1b64      	subs	r4, r4, r5
 80002c6:	10a4      	asrs	r4, r4, #2
 80002c8:	2600      	movs	r6, #0
 80002ca:	42a6      	cmp	r6, r4
 80002cc:	d105      	bne.n	80002da <__libc_init_array+0x2e>
 80002ce:	bd70      	pop	{r4, r5, r6, pc}
 80002d0:	f855 3b04 	ldr.w	r3, [r5], #4
 80002d4:	4798      	blx	r3
 80002d6:	3601      	adds	r6, #1
 80002d8:	e7ee      	b.n	80002b8 <__libc_init_array+0xc>
 80002da:	f855 3b04 	ldr.w	r3, [r5], #4
 80002de:	4798      	blx	r3
 80002e0:	3601      	adds	r6, #1
 80002e2:	e7f2      	b.n	80002ca <__libc_init_array+0x1e>
 80002e4:	0800030c 	.word	0x0800030c
 80002e8:	0800030c 	.word	0x0800030c
 80002ec:	0800030c 	.word	0x0800030c
 80002f0:	08000310 	.word	0x08000310

080002f4 <_init>:
 80002f4:	b5f8      	push	{r3, r4, r5, r6, r7, lr}
 80002f6:	bf00      	nop
 80002f8:	bcf8      	pop	{r3, r4, r5, r6, r7}
 80002fa:	bc08      	pop	{r3}
 80002fc:	469e      	mov	lr, r3
 80002fe:	4770      	bx	lr

08000300 <_fini>:
 8000300:	b5f8      	push	{r3, r4, r5, r6, r7, lr}
 8000302:	bf00      	nop
 8000304:	bcf8      	pop	{r3, r4, r5, r6, r7}
 8000306:	bc08      	pop	{r3}
 8000308:	469e      	mov	lr, r3
 800030a:	4770      	bx	lr
